BL51 BANKED LINKER/LOCATER V6.22.2.0                                                    12/15/2022  10:27:16  PAGE 1


BL51 BANKED LINKER/LOCATER V6.22.2.0, INVOKED BY:
C:\KEIL_V5\C51\BIN\BL51.EXE .\Release\system_FE81001.obj, .\Release\STARTUP.obj, .\Release\main.obj TO .\Release\Sample_
>> DrvLCM REGFILE (.\Release\Sample_DrvLCM.ORC) PRINT (.\Sample_DrvLCM.m51) RAMSIZE (256) CODE (0X0000-0X1FFF) XDATA (0X
>> 8000-0X87FF)


MEMORY MODEL: SMALL


INPUT MODULES INCLUDED:
  .\Release\system_FE81001.obj (SYSTEM_FE81001)
  .\Release\STARTUP.obj (?C_STARTUP)
  .\Release\main.obj (MAIN)
  C:\KEIL_V5\C51\LIB\C51S.LIB (?C?CCASE)
  C:\KEIL_V5\C51\LIB\C51S.LIB (?C_IBP)


LINK MAP OF MODULE:  .\Release\Sample_DrvLCM (SYSTEM_FE81001)


            TYPE    BASE      LENGTH    RELOCATION   SEGMENT NAME
            -----------------------------------------------------

            * * * * * * *   D A T A   M E M O R Y   * * * * * * *
            REG     0000H     0008H     ABSOLUTE     "REG BANK 0"
            DATA    0008H     0006H     UNIT         ?DT?_DELAY?MAIN
            DATA    000EH     0001H     UNIT         ?DT?LCMINIT?MAIN
            DATA    000FH     0001H     UNIT         ?DT?_DIG1?MAIN
            DATA    0010H     0001H     UNIT         ?DT?_DIG2?MAIN
            DATA    0011H     0001H     UNIT         ?DT?_DIG3?MAIN
            DATA    0012H     0001H     UNIT         ?DT?_DIG4?MAIN
            DATA    0013H     0001H     UNIT         ?DT?MAIN?MAIN
            DATA    0014H     0001H     UNIT         ?C?LIB_DATA
            IDATA   0015H     0001H     UNIT         ?STACK

            * * * * * * *   C O D E   M E M O R Y   * * * * * * *
            CODE    0000H     0003H     ABSOLUTE     
            CODE    0003H     0177H     UNIT         ?PR?IOCTRL?MAIN
            CODE    017AH     00A9H     UNIT         ?PR?_DIG1?MAIN
            CODE    0223H     00A9H     UNIT         ?PR?_DIG2?MAIN
            CODE    02CCH     00A9H     UNIT         ?PR?_DIG3?MAIN
            CODE    0375H     00A9H     UNIT         ?PR?_DIG4?MAIN
            CODE    041EH     003BH     UNIT         ?PR?_DELAY?MAIN
            CODE    0459H     003BH     UNIT         ?PR?MAIN?MAIN
            CODE    0494H     0036H     UNIT         ?PR?LCMINIT?MAIN
            CODE    04CAH     0026H     UNIT         ?C?LIB_CODE
            CODE    04F0H     001DH     UNIT         ?C_C51STARTUP
            CODE    050DH     000DH     UNIT         ?PR?LCM_CONFIG?MAIN
            CODE    051AH     000CH     UNIT         ?PR?POINT?MAIN
            CODE    0526H     0001H     UNIT         ?PR?SYSTEMINIT?SYSTEM_FE81001



OVERLAY MAP OF MODULE:   .\Release\Sample_DrvLCM (SYSTEM_FE81001)


SEGMENT
  +--> CALLED SEGMENT
BL51 BANKED LINKER/LOCATER V6.22.2.0                                                  12/15/2022  10:27:16  PAGE 2


---------------------
?C_C51STARTUP
  +--> ?PR?MAIN?MAIN

?PR?MAIN?MAIN
  +--> ?PR?LCM_CONFIG?MAIN
  +--> ?PR?_DIG1?MAIN
  +--> ?PR?_DIG2?MAIN
  +--> ?PR?POINT?MAIN
  +--> ?PR?_DIG3?MAIN
  +--> ?PR?_DIG4?MAIN
  +--> ?PR?_DELAY?MAIN

?PR?LCM_CONFIG?MAIN
  +--> ?PR?IOCTRL?MAIN
  +--> ?PR?LCMINIT?MAIN



SYMBOL TABLE OF MODULE:  .\Release\Sample_DrvLCM (SYSTEM_FE81001)

  VALUE           TYPE          NAME
  ----------------------------------

  -------         MODULE        SYSTEM_FE81001
  C:0000H         SYMBOL        _ICE_DUMMY_
  C:0526H         PUBLIC        SystemInit
  -------         PROC          SYSTEMINIT
  C:0526H         LINE#         38
  C:0526H         LINE#         39
  C:0526H         LINE#         41
  -------         ENDPROC       SYSTEMINIT
  -------         ENDMOD        SYSTEM_FE81001

  -------         MODULE        ?C_STARTUP
  C:04F0H         SEGMENT       ?C_C51STARTUP
  I:0015H         SEGMENT       ?STACK
  C:0000H         PUBLIC        ?C_STARTUP
  D:00E0H         SYMBOL        ACC
  D:00F0H         SYMBOL        B
  D:0083H         SYMBOL        DPH
  D:0082H         SYMBOL        DPL
  N:0001H         SYMBOL        IBPSTACK
  N:0100H         SYMBOL        IBPSTACKTOP
  N:0080H         SYMBOL        IDATALEN
  C:04F3H         SYMBOL        IDATALOOP
  N:0000H         SYMBOL        PBPSTACK
  N:0100H         SYMBOL        PBPSTACKTOP
  N:0000H         SYMBOL        PDATALEN
  N:0000H         SYMBOL        PDATASTART
  N:0000H         SYMBOL        PPAGE
  N:0000H         SYMBOL        PPAGEENABLE
  D:00A0H         SYMBOL        PPAGE_SFR
  D:0081H         SYMBOL        SP
  C:04F0H         SYMBOL        STARTUP1
  N:0000H         SYMBOL        XBPSTACK
  N:0000H         SYMBOL        XBPSTACKTOP
BL51 BANKED LINKER/LOCATER V6.22.2.0                                                  12/15/2022  10:27:16  PAGE 3


  N:0800H         SYMBOL        XDATALEN
  C:04FEH         SYMBOL        XDATALOOP
  N:8000H         SYMBOL        XDATASTART
  C:0000H         LINE#         126
  C:04F0H         LINE#         133
  C:04F2H         LINE#         134
  C:04F3H         LINE#         135
  C:04F4H         LINE#         136
  C:04F6H         LINE#         140
  C:04F9H         LINE#         141
  C:04FBH         LINE#         145
  C:04FDH         LINE#         147
  C:04FEH         LINE#         148
  C:04FFH         LINE#         149
  C:0500H         LINE#         150
  C:0502H         LINE#         151
  C:0504H         LINE#         170
  C:0507H         LINE#         185
  C:050AH         LINE#         196
  -------         ENDMOD        ?C_STARTUP

  -------         MODULE        MAIN
  C:0000H         SYMBOL        _ICE_DUMMY_
  D:0090H         PUBLIC        P1
  D:00B0H         PUBLIC        P3
  D:00A8H         PUBLIC        IE
  C:041EH         PUBLIC        _delay
  C:050DH         PUBLIC        LCM_Config
  D:00B8H         PUBLIC        IP
  C:0459H         PUBLIC        main
  C:051AH         PUBLIC        point
  C:0003H         PUBLIC        IOCtrl
  D:0098H         PUBLIC        SCON
  D:0088H         PUBLIC        TCON
  C:017AH         PUBLIC        _Dig1
  C:0223H         PUBLIC        _Dig2
  C:02CCH         PUBLIC        _Dig3
  C:0375H         PUBLIC        _Dig4
  D:00C8H         PUBLIC        T2CON
  C:0494H         PUBLIC        LCMInit
  D:00D0H         PUBLIC        PSW
  -------         PROC          _DELAY
  D:0008H         SYMBOL        cnt
  -------         DO            
  D:000AH         SYMBOL        i
  D:000CH         SYMBOL        j
  -------         ENDDO         
  C:041EH         LINE#         34
  C:0422H         LINE#         35
  C:0422H         LINE#         38
  C:0433H         LINE#         39
  C:0458H         LINE#         41
  -------         ENDPROC       _DELAY
  -------         PROC          LCMINIT
  -------         DO            
  D:000EH         SYMBOL        i
  -------         ENDDO         
BL51 BANKED LINKER/LOCATER V6.22.2.0                                                  12/15/2022  10:27:16  PAGE 4


  C:0494H         LINE#         53
  C:0494H         LINE#         54
  C:0494H         LINE#         58
  C:049FH         LINE#         61
  C:04A5H         LINE#         64
  C:04B7H         LINE#         65
  C:04C5H         LINE#         66
  C:04C9H         LINE#         67
  -------         ENDPROC       LCMINIT
  -------         PROC          IOCTRL
  C:0003H         LINE#         77
  C:0003H         LINE#         78
  C:0003H         LINE#         80
  C:000EH         LINE#         83
  C:002FH         LINE#         86
  C:0050H         LINE#         89
  C:0071H         LINE#         92
  C:0087H         LINE#         95
  C:009DH         LINE#         98
  C:00B3H         LINE#         101
  C:00C9H         LINE#         104
  C:00DFH         LINE#         107
  C:00F5H         LINE#         110
  C:010BH         LINE#         113
  C:0121H         LINE#         116
  C:0137H         LINE#         119
  C:014DH         LINE#         122
  C:0163H         LINE#         125
  C:0179H         LINE#         127
  -------         ENDPROC       IOCTRL
  -------         PROC          LCM_CONFIG
  C:050DH         LINE#         129
  C:050DH         LINE#         130
  C:050DH         LINE#         131
  C:0510H         LINE#         133
  C:0513H         LINE#         135
  C:0519H         LINE#         136
  -------         ENDPROC       LCM_CONFIG
  -------         PROC          _DIG1
  D:000FH         SYMBOL        num
  C:017AH         LINE#         138
  C:017CH         LINE#         139
  C:017CH         LINE#         140
  C:01A3H         LINE#         141
  C:01A3H         LINE#         143
  C:01A3H         LINE#         144
  C:01A9H         LINE#         145
  C:01AFH         LINE#         146
  C:01B0H         LINE#         148
  C:01B0H         LINE#         149
  C:01B5H         LINE#         150
  C:01BBH         LINE#         151
  C:01BCH         LINE#         153
  C:01BCH         LINE#         154
  C:01C2H         LINE#         155
  C:01C8H         LINE#         156
  C:01C9H         LINE#         158
BL51 BANKED LINKER/LOCATER V6.22.2.0                                                  12/15/2022  10:27:16  PAGE 5


  C:01C9H         LINE#         159
  C:01CFH         LINE#         160
  C:01D5H         LINE#         161
  C:01D6H         LINE#         163
  C:01D6H         LINE#         164
  C:01DCH         LINE#         165
  C:01E2H         LINE#         166
  C:01E3H         LINE#         168
  C:01E3H         LINE#         169
  C:01E9H         LINE#         170
  C:01EFH         LINE#         171
  C:01F0H         LINE#         173
  C:01F0H         LINE#         174
  C:01F6H         LINE#         175
  C:01FCH         LINE#         176
  C:01FDH         LINE#         178
  C:01FDH         LINE#         179
  C:0202H         LINE#         180
  C:0208H         LINE#         181
  C:0209H         LINE#         183
  C:0209H         LINE#         184
  C:020FH         LINE#         185
  C:0215H         LINE#         186
  C:0216H         LINE#         188
  C:0216H         LINE#         189
  C:021CH         LINE#         190
  C:0222H         LINE#         191
  C:0222H         LINE#         193
  C:0222H         LINE#         195
  -------         ENDPROC       _DIG1
  -------         PROC          _DIG2
  D:0010H         SYMBOL        num
  C:0223H         LINE#         196
  C:0225H         LINE#         197
  C:0225H         LINE#         198
  C:024CH         LINE#         199
  C:024CH         LINE#         201
  C:024CH         LINE#         202
  C:0252H         LINE#         203
  C:0258H         LINE#         204
  C:0259H         LINE#         206
  C:0259H         LINE#         207
  C:025EH         LINE#         208
  C:0264H         LINE#         209
  C:0265H         LINE#         211
  C:0265H         LINE#         212
  C:026BH         LINE#         213
  C:0271H         LINE#         214
  C:0272H         LINE#         216
  C:0272H         LINE#         217
  C:0278H         LINE#         218
  C:027EH         LINE#         219
  C:027FH         LINE#         221
  C:027FH         LINE#         222
  C:0285H         LINE#         223
  C:028BH         LINE#         224
  C:028CH         LINE#         226
BL51 BANKED LINKER/LOCATER V6.22.2.0                                                  12/15/2022  10:27:16  PAGE 6


  C:028CH         LINE#         227
  C:0292H         LINE#         228
  C:0298H         LINE#         229
  C:0299H         LINE#         231
  C:0299H         LINE#         232
  C:029FH         LINE#         233
  C:02A5H         LINE#         234
  C:02A6H         LINE#         236
  C:02A6H         LINE#         237
  C:02ABH         LINE#         238
  C:02B1H         LINE#         239
  C:02B2H         LINE#         241
  C:02B2H         LINE#         242
  C:02B8H         LINE#         243
  C:02BEH         LINE#         244
  C:02BFH         LINE#         246
  C:02BFH         LINE#         247
  C:02C5H         LINE#         248
  C:02CBH         LINE#         249
  C:02CBH         LINE#         251
  C:02CBH         LINE#         253
  -------         ENDPROC       _DIG2
  -------         PROC          _DIG3
  D:0011H         SYMBOL        num
  C:02CCH         LINE#         254
  C:02CEH         LINE#         255
  C:02CEH         LINE#         256
  C:02F5H         LINE#         257
  C:02F5H         LINE#         259
  C:02F5H         LINE#         260
  C:02FBH         LINE#         261
  C:0301H         LINE#         262
  C:0302H         LINE#         264
  C:0302H         LINE#         265
  C:0307H         LINE#         266
  C:030DH         LINE#         267
  C:030EH         LINE#         269
  C:030EH         LINE#         270
  C:0314H         LINE#         271
  C:031AH         LINE#         272
  C:031BH         LINE#         274
  C:031BH         LINE#         275
  C:0321H         LINE#         276
  C:0327H         LINE#         277
  C:0328H         LINE#         279
  C:0328H         LINE#         280
  C:032EH         LINE#         281
  C:0334H         LINE#         282
  C:0335H         LINE#         284
  C:0335H         LINE#         285
  C:033BH         LINE#         286
  C:0341H         LINE#         287
  C:0342H         LINE#         289
  C:0342H         LINE#         290
  C:0348H         LINE#         291
  C:034EH         LINE#         292
  C:034FH         LINE#         294
BL51 BANKED LINKER/LOCATER V6.22.2.0                                                  12/15/2022  10:27:16  PAGE 7


  C:034FH         LINE#         295
  C:0354H         LINE#         296
  C:035AH         LINE#         297
  C:035BH         LINE#         299
  C:035BH         LINE#         300
  C:0361H         LINE#         301
  C:0367H         LINE#         302
  C:0368H         LINE#         304
  C:0368H         LINE#         305
  C:036EH         LINE#         306
  C:0374H         LINE#         307
  C:0374H         LINE#         309
  C:0374H         LINE#         310
  -------         ENDPROC       _DIG3
  -------         PROC          _DIG4
  D:0012H         SYMBOL        num
  C:0375H         LINE#         311
  C:0377H         LINE#         312
  C:0377H         LINE#         313
  C:039EH         LINE#         314
  C:039EH         LINE#         316
  C:039EH         LINE#         317
  C:03A4H         LINE#         318
  C:03AAH         LINE#         319
  C:03ABH         LINE#         321
  C:03ABH         LINE#         322
  C:03B0H         LINE#         323
  C:03B6H         LINE#         324
  C:03B7H         LINE#         326
  C:03B7H         LINE#         327
  C:03BDH         LINE#         328
  C:03C3H         LINE#         329
  C:03C4H         LINE#         331
  C:03C4H         LINE#         332
  C:03CAH         LINE#         333
  C:03D0H         LINE#         334
  C:03D1H         LINE#         336
  C:03D1H         LINE#         337
  C:03D7H         LINE#         338
  C:03DDH         LINE#         339
  C:03DEH         LINE#         341
  C:03DEH         LINE#         342
  C:03E4H         LINE#         343
  C:03EAH         LINE#         344
  C:03EBH         LINE#         346
  C:03EBH         LINE#         347
  C:03F1H         LINE#         348
  C:03F7H         LINE#         349
  C:03F8H         LINE#         351
  C:03F8H         LINE#         352
  C:03FDH         LINE#         353
  C:0403H         LINE#         354
  C:0404H         LINE#         356
  C:0404H         LINE#         357
  C:040AH         LINE#         358
  C:0410H         LINE#         359
  C:0411H         LINE#         361
BL51 BANKED LINKER/LOCATER V6.22.2.0                                                  12/15/2022  10:27:16  PAGE 8


  C:0411H         LINE#         362
  C:0417H         LINE#         363
  C:041DH         LINE#         364
  C:041DH         LINE#         366
  C:041DH         LINE#         368
  -------         ENDPROC       _DIG4
  -------         PROC          POINT
  C:051AH         LINE#         370
  C:051AH         LINE#         371
  C:051AH         LINE#         372
  C:0525H         LINE#         373
  -------         ENDPROC       POINT
  -------         PROC          MAIN
  -------         DO            
  D:0013H         SYMBOL        i
  -------         ENDDO         
  C:0459H         LINE#         384
  C:0459H         LINE#         385
  C:0459H         LINE#         386
  C:045CH         LINE#         388
  C:045FH         LINE#         390
  C:045FH         LINE#         391
  C:045FH         LINE#         393
  C:0464H         LINE#         394
  C:0469H         LINE#         395
  C:046CH         LINE#         396
  C:0471H         LINE#         397
  C:0476H         LINE#         398
  C:047DH         LINE#         400
  C:047FH         LINE#         401
  C:0491H         LINE#         402
  -------         ENDPROC       MAIN
  -------         ENDMOD        MAIN

  -------         MODULE        ?C?CCASE
  C:04CAH         PUBLIC        ?C?CCASE
  -------         ENDMOD        ?C?CCASE

  -------         MODULE        ?C_IBP
  D:0014H         PUBLIC        ?C_IBP
  -------         ENDMOD        ?C_IBP



FUNCTION REGISTER MASKS


FUNCTION . . . REG MASK
-----------------------

IOCTRL . . . . @0xe301
LCMINIT. . . . @0xf303
LCM_CONFIG . . @0xf303
MAIN . . . . . @0xf383
POINT. . . . . @0xe301
SYSTEMINIT . . @0x8000
_DELAY . . . . @0xf000
BL51 BANKED LINKER/LOCATER V6.22.2.0                                                  12/15/2022  10:27:16  PAGE 9


_DIG1. . . . . @0xf380
_DIG2. . . . . @0xf380
_DIG3. . . . . @0xf380
_DIG4. . . . . @0xf380

*** WARNING L16: UNCALLED SEGMENT, IGNORED FOR OVERLAY PROCESS
    SEGMENT: ?PR?SYSTEMINIT?SYSTEM_FE81001

Program Size: data=22.0 xdata=0 code=1319
LINK/LOCATE RUN COMPLETE.  1 WARNING(S),  0 ERROR(S)
